:020000040000FA
:040000006B303A28FF
:08000800A000030EA100831209
:100010008B1C32288B1031181428B11C3228643004
:10002000010203183128182800001628172818285C
:1000300019281A281B281C281D281E281F283110A3
:10004000B114A810031005190314AA0DA90DA80DC9
:10005000B00B322831152A08AF002908AE00280855
:10006000AD00B11081010B11210E8300A00E200EF6
:02007000090085
:0C007400203084008001840A6030040207
:10008000031C3C281230B000A42183160C308505D7
:1000900087018312850187010730990000309A009B
:1000A000103083168E008312603083168F00831207
:1000B0000030831691008312C830831681008312AA
:1000C00031309000003083168C00831210308B008A
:1000D000831600309B001C141A088312BC00831680
:1000E00010309B001C141A088312BD00E821810106
:1000F0008E018F010B118B100B108C018B178E2032
:100100003119A420B30B8C28031085190314B90DE1
:10011000F03039020319292101227F2864003118A7
:1001200008000B1D08000B11B11031141230B00083
:10013000051D9F2832148316011383120800321004
:10014000831601178312080031110130B7008B1399
:100150002030370783169B001C141A088312A40052
:10016000A500C030A5061030370783169B001C146D
:100170001A088312A3000030370783169B001C1453
:100180001A088312A2008B17321CCC2822090339CB
:10019000A200A309A409A50922082D02031D2329F1
:1001A00023082E02031D232924082F02031DFB28E8
:1001B00001303702031DDF283D143E14B121023007
:1001C0003702031DE628BD143E14B5210330370263
:1001D000031DED283D153E14B92104303702031DDF
:1001E000F428BD153E14BD2105303702031DFB2840
:1001F0003D163E14C12125082F02031D232901307D
:100200003702031D06293D103E14C5210230370276
:10021000031D0D29BD103E14C92103303702031DF3
:1002200014293D113E14CD2104303702031D1B2932
:10023000BD113E14D12105303702031D22293D1284
:100240003E14D5212329B70A0630370203180800C7
:10025000A7280130B600B300B400B500B70085018F
:100260008701B1138E20B30B552903108519031490
:10027000B90DF030390203197C29B40B552901302E
:1002800037020319D921023037020319DC21033068
:1002900037020319DF21043037020319E221053048
:1002A00037020319E5219630B400311D322931118E
:1002B000321C5F292D090339AD00AE09AF092F1C8F
:1002C000B1132F1C3229B11B32292E183229B11734
:1002D0008B1320303707BB002F08BA008F21103056
:1002E0003707BB002E08BA008F2100303707BB004C
:1002F0002D08BA008F218B1785018701B70AB60137
:1003000006303702031C3229E82108003E1C080091
:100310003E101030BB003D08BA008F2108008B133F
:100320003A0883161C159A0083123B0883169B001B
:1003300055309D00AA309D009C1464009C189D2996
:100340001C1183128B170800FF30D000D415D5156F
:10035000D615D715D815D915DA15DB15DC15DD1529
:100360000800D2104E14CE100800D2114E15CE1136
:100370000800D2124E16CE120800D2134E17CE131A
:100380000800D3104F14CF1008005210CE144E1096
:1003900008005211CE154E1108005212CE164E1200
:1003A00008005213CE174E1308005310CF144F10ED
:1003B0000800303085060800033085060800063046
:1003C00087060800213087060800183087060800D5
:1003D0003D184E143D1CCE14BD184E15BD1CCE1537
:1003E0003D194E163D1DCE16BD194E17BD1DCE171B
:1003F0003D1A4F143D1ECF144E08D200CF00D3003B
:1004000008008F08031908008F01D00F432BD00A72
:10041000521C192A541D0F2AD4015416272AD41D00
:10042000142AD4015416272A541E272AD401D4147E
:10043000272AD41C1E2AD4015415272A541D232AE6
:10044000D401D415272A541E272AD4015415D21CAE
:10045000382A551D2E2AD5015516462AD51D332A70
:10046000D5015516462A551E462AD501D514462AC9
:10047000D51C3D2AD5015515462A551D422AD501C0
:10048000D515462A551E462AD5015515521D572AFF
:10049000561D4D2AD6015616652AD61D522AD6015A
:1004A0005616652A561E652AD601D614652AD61C0C
:1004B0005C2AD6015615652A561D612AD601D61525
:1004C000652A561E652AD6015615D21D762A571D55
:1004D0006C2AD7015716842AD71D712AD7015716BF
:1004E000842A571E842AD701D714842AD71C7B2A32
:1004F000D7015715842A571D802AD701D715842A7A
:10050000571E842AD7015715521E952A581D8B2A2B
:10051000D8015816A32AD81D902AD8015816A32A04
:10052000581EA32AD801D814A32AD81C9A2AD80165
:100530005815A32A581D9F2AD801D815A32A581E3A
:10054000A32AD8015815D21EB42A591DAA2AD901A6
:100550005916C22AD91DAF2AD9015916C22A591EC5
:10056000C22AD901D914C22AD91CB92AD9015915CC
:10057000C22A591DBE2AD901D915C22A591EC22A1A
:10058000D9015915521FD32A5A1DC92ADA015A1600
:10059000E12ADA1DCE2ADA015A16E12A5A1EE12A88
:1005A000DA01DA14E12ADA1CD82ADA015A15E12A2A
:1005B0005A1DDD2ADA01DA15E12A5A1EE12ADA018A
:1005C0005A15D21FF22A5B1DE82ADB015B16002BAD
:1005D000DB1DED2ADB015B16002B5B1E002BDB0114
:1005E000DB14002BDB1CF72ADB015B15002B5B1DEA
:1005F000FC2ADB01DB15002B5B1E002BDB015B15EE
:10060000531C112B5C1D072BDC015C161F2BDC1D02
:100610000C2BDC015C161F2B5C1E1F2BDC01DC1479
:100620001F2BDC1C162BDC015C151F2B5C1D1B2BF0
:10063000DC01DC151F2B5C1E1F2BDC015C15D31CA1
:10064000302B5D1D262BDD015D163E2BDD1D2B2B7A
:10065000DD015D163E2B5D1E3E2BDD01DD143E2BC4
:10066000DD1C352BDD015D153E2B5D1D3A2BDD01BB
:10067000DD153E2B5D1E3E2BDD015D1586214E08EE
:10068000D2004F08D3005008D1000C305405031D90
:1006900005120C305505031D85120C305605031D3F
:1006A00005100C305705031D85100C305805031D2F
:1006B00087100C305905031D07110C305A05031D16
:1006C00007100C305B05031D87120C305C05031D01
:1006D00007120C305D05031D871151080E02031827
:1006E0009D2B12305405031D051612305505031DB0
:1006F000851612305605031D051412305705031DCB
:10070000851412305805031D871412305905031D36
:10071000071512305A05031D071412305B05031D1F
:10072000871612305C05031D071612305D05031D88
:100730008715FF305002031908008F08031D0800B9
:100740008E2051080E02031C9D2B18305405031DEA
:10075000051206305405031D051618305505031DF6
:10076000851206305505031D851618305605031DE4
:10077000051006305605031D051418305705031DD6
:10078000851006305705031D851418305805031DC4
:10079000871006305805031D871418305905031DAE
:1007A000071106305905031D071518305A05031D9A
:1007B000071006305A05031D071418305B05031D8A
:1007C000871206305B05031D871618305C05031D74
:1007D000071206305C05031D071618305D05031D62
:0C07E000871106305D05031D8715080019
:084000000200030002000600AB
:02400E00CC33B1
:10420000010003000300030003000200020002009B
:1042100002000000000000000000FF00FF00FF009F
:10422000000000000000000000000000000000008E
:104230000000C000C000C000C000FF00FF00FF0081
:104240000100C300F300CF00FF00C300F300CF0064
:10425000FF00C300F300CF00FF00FF00FF00FF00DE
:10426000FF00FF00FF00FF00FF00FF00FF00FF0056
:10427000FF00FF00FF00FF00FF00FF00FF00FF0046
:10428000FF00FF00FF00FF00FF00FF00FF00FF0036
:10429000FF00FF00FF00FF00FF00FF00FF00FF0026
:1042A000FF00FF00FF00FF00FF00FF00FF00FF0016
:1042B000FF00FF00FF00FF00FF00FF00FF00FF0006
:1042C000FF00FF00FF00FF00FF00FF00FF00FF00F6
:1042D000FF00FF00FF00FF00FF00FF00FF00FF00E6
:1042E000FF00FF00FF00FF00FF00FF00FF00FF00D6
:1042F000FF00FF00FF00FF00FF00FF00FF00AA001B
:00000001FF
